:020000021000EC
:10F800000C9446FC0C9463FC0C9463FC0C9463FC19
:10F810000C9463FC0C9463FC0C9463FC0C9463FCEC
:10F820000C9463FC0C9463FC0C9463FC0C9463FCDC
:10F830000C9463FC0C9463FC0C9463FC0C9463FCCC
:10F840000C9463FC0C9463FC0C9463FC0C9463FCBC
:10F850000C9463FC0C9463FC0C9463FC0C9463FCAC
:10F860000C9463FC0C9463FC0C9463FC0C9463FC9C
:10F870000C9463FC0C9463FC0C9463FC0C9463FC8C
:10F880000C9463FC0C9463FC0C9463FC11241FBE69
:10F89000CFEFD0E1DEBFCDBF11E0A0E0B1E0EEE5FB
:10F8A000FFEF01E00BBF02C007900D92A030B1073F
:10F8B000D9F712E0A0E0B1E001C01D92A434B10775
:10F8C000E1F70C9471FF0C9400FC0F92AF93BF937F
:10F8D000CF93DF93EF93FF93FC01EA01DB01D8950F
:10F8E000099231961197D9F7FF91EF91DF91CF915E
:10F8F000BF91AF910F9008950F921F920F931F9396
:10F90000AF93BF93CF93DF93EF93FF93FC01EA0193
:10F91000DB0110E00990199001E04CD0329612976B
:10F9200011F01250B9F7FC0103E044D005E042D0D9
:10F9300000E011E0800F911F109759F7FF91EF91B0
:10F94000DF91CF91BF91AF911F910F911F900F90B9
:10F9500008950F931F93EF93FF93FC0103E02AD0C8
:10F9600000E011E0E00FF11FE617F707B9F7FF918C
:10F97000EF911F910F9108950F930F9222D0082EAF
:10F9800009E018D00F900F9108950F930F92EF9305
:10F99000FF9317D0FC0160936800C895802DFF91FC
:10F9A000EF910F900F9108950F930BD001E102D0CA
:10F9B0000F910895E199FECF00936800E895FFFF4D
:10F9C00000000091680000FDFCCF089588E089B92F
:10F9D0008AB188618AB908958AB1877E8AB9089503
:10F9E0008CB95E9BFECF5E9A08958CB199270895DD
:10F9F0008BB19927807890700895EF92FF920F93C2
:10FA00001F93CF93DF937B01C0E0D0E0C617D707E9
:10FA100070F48C010E94F8FC8823E1F30E94F5FC4D
:10FA2000F80181938F012196CE15DF0598F381E0CF
:10FA300090E0DF91CF911F910F91FF90EF9008958B
:10FA4000EF92FF920F931F93CF93DF937C018B0173
:10FA5000C0E0D0E0C017D10738F4F70181917F01F1
:10FA60000E94F0FC2196F6CF81E090E0DF91CF91EB
:10FA70001F910F91FF90EF90089540E050E04817DC
:10FA8000590750F42FEC37E000002150304037FF89
:10FA9000FBCF4F5F5F4FF3CF08950E94ECFC0E94B5
:10FAA000000008950E94F8FC8823E1F30E94F5FC11
:10FAB000803219F481E090E0089585E10E94F0FC25
:10FAC00080E090E0089590E0282F33272138310519
:10FAD00089F02238310524F42038310549F00DC071
:10FAE0002238310549F02839310539F493E005C051
:10FAF00092E003C091E001C092E1892F9927089517
:10FB000040E050E060914001709141014617570775
:10FB1000D0F42091420230914302E2E4F1E03FBB95
:10FB20002EBB2F5F3F4F80818DBBE29AE19AE19916
:10FB3000FECF4F5F5F4F31964617570780F33093E4
:10FB4000430220934202089540E050E0609140015A
:10FB50007091410146175707B0F42091420230914D
:10FB60004302E2E4F1E03FBB2EBB2F5F3F4FE09A40
:10FB70008DB381934F5F5F4F46175707A0F33093C4
:10FB80004302209342020895CF93DF938091420273
:10FB90009091430297FF03C081E08BBF01C01BBE61
:10FBA000C0E0D0E08091400190914101C817D90791
:10FBB000A0F4CE018E5B9E4F209142023091430211
:10FBC000220F331FAC0160E071E0C9018C0F9D1F53
:10FBD0000E947CFCC050DF4FE5CF0E94D4FCDF9137
:10FBE000CF910895209142023091430237FF03C024
:10FBF00081E08BBF01C01BBE42E451E06091400137
:10FC000070914101C901880F991F0E9465FC0895F8
:10FC1000CF93C0E069E081E090E00E94C5FC9927A5
:10FC200084FF03C08F7E0E94BCFC0E94F8FC8823E6
:10FC3000E1F30E94F5FC9927823591051CF580358A
:10FC400091050CF05CC08134910509F462C08234E6
:10FC500091057CF481339105B1F18233910524F44F
:10FC6000C09709F44CC037C18034910509F437C1FD
:10FC700032C18234910509F45FC08534910509F4DD
:10FC80005EC029C18635910509F4F0C0873591051C
:10FC90004CF48235910509F45FC08535910509F46E
:10FCA00068C019C18437910509F4A3C0853791054F
:10FCB0002CF48436910509F475C00DC18537910582
:10FCC00009F4C4C008C10E9452FD882309F4ADCFD5
:10FCD00084E10E94F0FC81E40E94F0FC86E50E9431
:10FCE000F0FC82E50E94F0FC80E20E94F0FC83E5DB
:10FCF0000E94F0FC84E50E94F0FC8BE406C00E94A8
:10FD000052FD882309F491CF84E10E94F0FC80E148
:10FD1000E3C061E070E080E091E00E94FDFC0E94A1
:10FD200052FD882309F481CF84E10E94F0FC809188
:10FD300000010E9463FDE9CF64E170E008C061E06A
:10FD400070E080E091E00E94FDFC64E070E080E003
:10FD500091E00E94FDFCD3CF0E9452FD882309F45C
:10FD600064CF60E070E0CB010E94A9FC0E94D4FC4B
:10FD7000CBCF62E070E080E091E00E94FDFC0E9449
:10FD800052FD882309F451CF209100018091010197
:10FD90009927982F8827820F911D90934302809373
:10FDA0004202B2CF63E070E080E091E00E94FDFC8F
:10FDB00020910101809100019927982F8827820FB7
:10FDC000911D9093410180934001BC0182E491E038
:10FDD0000E94FDFC0E9452FD882309F426CF8091E9
:10FDE0000201863419F40E94C4FD8ECF0E9480FD6A
:10FDF0008BCF63E070E080E091E00E94FDFC2091F9
:10FE00000101809100019927982F8827820F911D69
:10FE100090934101809340010E9452FD882309F490
:10FE200004CF80910201863419F40E94F2FD02C0D1
:10FE30000E94A4FD84E10E94F0FC60914001709159
:10FE4000410182E491E00E9420FD61CF0E9452FDB9
:10FE5000882309F4EACE84E10E94F0FC8EE10E943E
:10FE6000F0FC87E90E94F0FC82E04FCF64E070E094
:10FE700080E091E00E94FDFC0E9452FD882309F47D
:10FE8000D4CE84E10E94F0FC80910001803531F4F1
:10FE900080910101882361F4C82F17C0883531F49F
:10FEA00080910101883061F4C3E00FC0803531F4E6
:10FEB00080910101883049F4C2E007C0883529F4F7
:10FEC00080910101882309F4C1E069E08C2F992712
:10FED0000E94C5FC1ACF85E10E94F0FCA6CECF910E
:10FEE0000895CFEFD0E1DEBFCDBFCEE1F894AEEF05
:10FEF000BFE00E94A6FF802D843B79F4AFEFBFE006
:10FF00000E94A6FF802D833C41F4ADEFBFE00E942C
:10FF1000A6FF802D992780936F000E94E6FC0E9427
:10FF2000F5FC84E690E00E943DFD0E94F8FC8823E9
:10FF300019F00E9408FE04C0C150C8BBCC2389F749
:10FF40000E944DFD80E090E00C94AEFFE199FECF61
:0EFF5000BFBBAEBBE09A11960DB20895FFCF75
:040000031000F800F1
:00000001FF
